:020000000D28C9
:10000800FE00030EF3000A08F40083127F08F500CF
:100018006F290308A000BF29F229F529F829092A20
:040028000C2A0F2A65
:100200000029FF0001308A007F0882070629562A4C
:10021000532AA4291E22322203304F220030F0211B
:100220000030D821831205183229FE30A505FF3091
:10023000A605A705A8052808803A25042604270452
:10024000031D3D290230F0210130D821F430831202
:10025000AF000130B0000230B100B201B20A442256
:1002600085123D292514250A0319260A0319270A90
:100270007F3003192806031985160310A50DA60D56
:10028000A70DA80D85185E29FE30A105FF30A20537
:10029000A305A4052408803A210422042304031D95
:1002A00069290230F021F430AF000130B000013094
:1002B000B100B201B20A4422851269292114210A2F
:1002C0000319220A0319230A7F300319240603198C
:1002D00085160310A10DA20DA30DA40D12290B1953
:1002E0008B1E9B29FB08031D9229F60A0319F70AA6
:1002F0000319F80A0319F90A00307902031D8A2943
:1003000000307802031D8A2900307702031D8A29F4
:1003100006307602031C922904308506F601F701A7
:10032000F801F9017C08031997297C0801217A0852
:10033000831281000B117508FF0074088A00730E88
:100340008300FE0E7E0E09002C08F2002B08F1003F
:10035000AB0A0319AC0A2A087202031DB129290845
:100360007102031C08002E080319BC292E08012164
:1003700083122D0BBC29AE01AB01AC010800FF308C
:10038000F601F701F801F901A901AA01AB01AC01DD
:10039000AD01AE01A100A200A300A400A500A6002B
:1003A000A700A800B330FA000130FB0083010A293E
:1003B000AF00E729F53083168115FA000800B33045
:1003C00083160111811401148111FA0008002F080D
:1003D000003A0319DA29013A0319DF29EF29080045
:1003E000AF00FB29FB0105160800FB010512080000
:1003F000FB01FB0A08002F088400033004020318E5
:10040000080000308A001030040782000800F00065
:10041000122AFB0105160800FB0105120800FB016A
:10042000FB0A080070088400033004020318080067
:1004300000308A001330040782000800073099005A
:1004400015089F0183169F018113960105148514D9
:100450001514951405110512851283120511051244
:100460008516080083160F178F160F168F110F10A1
:10047000011181140114811181128B110B100B11C8
:100480008B168B170B170800AB01AC013008AA00C4
:100490002F08A9003108AE003208AD000800831211
:1004A000AF00FC00080001300722080000300722DE
:0204B000080042
:02400E00E4F0DC
:00000001FF
